:020000040800F2
:10000000A013002075060008250300082703000838
:100010002B0300082F030008330300080000000032
:10002000000000000000000000000000370300088E
:1000300039030008000000003B0300083D030008EE
:100040008F0600088F0600088F0600088F0600083C
:100050008F0600088F0600088F0600088F0600082C
:100060008F0600088F0600088F0600088F0600081C
:100070008F0600088F0600088F0600088F0600080C
:100080008F0600088F0600088F0600088F060008FC
:100090008F0600088F0600088F0600088F060008EC
:1000A0008F0600088F0600088F0600088F060008DC
:1000B0008F0600088F0600088F0600088F060008CC
:1000C0008F0600088F0600088F0600088F060008BC
:1000D0008F060008792300083D1E00088F060008DF
:1000E000C72500088F0600088F0600088F06000845
:1000F0008F0600088F0600088F0600088F0600088C
:100100008F0600088F0600088F0600088F0600087B
:100110008F0600088F0600088F0600088F0600086B
:100120008F0600088F0600088F0600088F0600085B
:100130008F0600088F0600088F0600088F0600084B
:100140008F0600088F0600088F0600088F0600083B
:100150008F0600088F0600088F0600088F0600082B
:100160008F0600088F0600088F0600088F0600081B
:100170008F0600088F0600088F0600088F0600080B
:100180008F0600088F06000800F002F800F044F81F
:100190000AA090E8000C82448344AAF10107DA45E2
:1001A00001D100F039F8AFF2090EBAE80F0013F0F0
:1001B000010F18BFFB1A43F001031847FC2700008A
:1001C0001C280000103A24BF78C878C1FAD852071A
:1001D00024BF30C830C144BF04680C6070470000C1
:1001E0000023002400250026103A28BF78C1FBD840
:1001F000520728BF30C148BF0B607047642902F026
:100200004982782902F08282002070471FB502F0EF
:10021000B9FB1FBD10B510BD02F081FB1146FFF701
:10022000F5FF00F039F802F09FFB03B4FFF7F2FF8F
:1002300003BC01F023FD000010B53648006841F210
:100240001001884210D100203349087001F00AFAE9
:100250000221102001F05AFA40F201112D4801F05C
:100260006EFB01F00CFA16E02A48006841F2111109
:10027000884203D10120284908700CE02548006815
:1002800040F20111884203D102202349087002E0A4
:1002900002202149087010BD00F0DCF9FFF7CCFF07
:1002A0004FF480611D4800F05DFB28BB4FF40061F6
:1002B0001A4800F057FBF8B94FF47A7000F0AAF929
:1002C0004FF48061154800F04DFBA8B94FF4006170
:1002D000124800F047FB78B901F0C4F90221102060
:1002E00001F014FA40F201110A4801F028FB01F074
:1002F000C6F90220084908700748007808B101F0E3
:1003000088FE06E000200649086001F020FF01F0A9
:100310009DFEF7E700800008000000200004024076
:1003200088824042704700BFFEE700BFFEE700BF83
:10033000FEE700BFFEE77047704770477047000058
:100340000CB50020019000907648006840F48030A1
:100350007449086000BF7348006800F400300090E2
:100360000198401C0190009818B90198B0F5A04F71
:10037000F1D16C48006800F4003010B10120009009
:1003800001E0002000900098012846D165484030E7
:10039000006840F08050634940310860624800685E
:1003A00040F44040604908605E48083000685D499C
:1003B000083108600846006840F4004008600846BC
:1003C000006840F4A05008605848091F0860081FE2
:1003D000006840F08070091F086000BF5148006845
:1003E00000F000700028F9D040F205705049086014
:1003F0004C480830006820F003004A490831086082
:100400000846006840F00200086000BF4548083018
:10041000006800F00C000828F8D10CBD10B5454864
:10042000006840F47000434908603E48006840F0AE
:1004300001003C49086000203A4908310860394809
:1004400000683D490840374908603C48091D08607C
:10045000081F006820F48020091F0860002031492F
:100460000C310860FFF76CFF4FF0006031498039B4
:10047000086010BD70B50020002202230024022174
:10048000284D08352D6805F00C0020B1042806D051
:10049000082834D107E02A4D2A4E356033E02A4D32
:1004A000284E35602FE01F4D2D1D2D68C5F380545B
:1004B0001C4D2D1D2D6805F03F0154B1224DB5FB9B
:1004C000F1F5184E361D3668C6F3881605FB06F2A0
:1004D00009E01B4DB5FBF1F5124E361D3668C6F32B
:1004E000881605FB06F20F4D2D1D2D68C5F301453D
:1004F0006D1C6B00B2FBF3F5124E356003E0104D3E
:10050000104E356000BF00BF064D08352D68C5F39D
:1005100003150E4E705D0B4D2D68C540094E3560BC
:1005200070BD0000003802400070004008544007D1
:10053000003C024088ED00E0FFFFF6FE1030002492
:100540000024F4000400002000127A0008000020BB
:1005500010B504466FF0040000F0FEF8E11704EB5C
:100560005171C1F3C701394A11701046007800EB90
:100570004001C1EBC0104FF6FF7101EAC0003449E1
:10058000088010BD0146314A12784A434FF0E023FB
:100590005A6100229A611A46126942F001021A61F8
:1005A00000BF4FF0E022106900F001021AB100F420
:1005B0008032002AF5D04FF0E022126922F00102C9
:1005C0004FF0E0231A6100229A6170470146204AE9
:1005D00012884A434FF0E0235A6100229A611A467A
:1005E000126942F001021A6100BF4FF0E022106967
:1005F00000F001021AB100F48032002AF5D04FF069
:10060000E022126922F001024FF0E0231A61002279
:100610009A61704770B504464FF4077094FBF0F090
:10062000C6B24FF4077094FBF0F100FB114085B2A5
:1006300005E04FF40770FFF7C9FF701EC6B2002E29
:10064000F7D115B12846FFF7C1FF70BD1800002093
:100650001A00002010B51020FFF77AFF4FF4E130A8
:1006600001F03DFB4FF4E13001F08FFB01F05AFF48
:1006700010BD00000948804709480047FEE7FEE733
:10068000FEE7FEE7FEE7FEE7FEE7FEE7FEE7FEE742
:1006900004480549054A064B704700001D04000840
:1006A00089010008A00D0020A0130020A00F002049
:1006B000A00F002032490143324A1160704770B5E3
:1006C000002100230F22C4781CB32E4C246804F4AC
:1006D000E064C4F5E064C4F30721C1F10404E3B2AB
:1006E0000A4144789C40E1B28478144021430C07CD
:1006F000210E254C05786155047804F01F0501246E
:10070000AC4005786D11AD0005F1E025C5F800415C
:1007100009E0047804F01F050124AC401B4D067865
:10072000761145F8264070BD194A0A400243154B20
:100730001B1F1A60704739B1124A121D126802431A
:10074000104B1B1D1A6006E00E4A121D12688243F0
:100750000C4B1B1D1A607047042808D14FF0E02194
:10076000096941F004014FF0E022116107E04FF008
:10077000E021096921F004014FF0E0221161704786
:100780000000FA050CED00E000E400E080E100E08C
:1007900080FFFF1F10B504469848844208D101210C
:1007A000084600F086FB0021012000F082FB76E085
:1007B0009348844208D10121022000F07AFB0021F5
:1007C000022000F076FB6AE08E48844208D10121C5
:1007D000042000F06EFB0021042000F06AFB5EE0C4
:1007E0008948844208D10121082000F062FB0021E1
:1007F000082000F05EFB52E08448844208D10121C9
:10080000102000F056FB0021102000F052FB46E0C3
:100810007F48844208D10121202000F04AFB0021BA
:10082000202000F046FB3AE07A48844208D10121BA
:10083000402000F03EFB0021402000F03AFB2EE07B
:100840007548844208D10121802000F032FB00214C
:10085000802000F02EFB22E07048844208D1012164
:10086000801500F026FB0021A01500F022FB16E009
:100870006B48844208D10121401500F01AFB002189
:10088000601500F016FB0AE06648844207D101219A
:10089000001500F00EFB0021201500F00AFB10BD32
:1008A000F0B50A4600210023002400BF3DE00125E9
:1008B00005FA01F3156805EA03049C4234D1056882
:1008C0004F000326BE40B543056015794E00B54084
:1008D0000668354305601579012D02D01579022D82
:1008E00016D185684F000326BE40B5438560557913
:1008F0004E00B540866835438560456801268E40C8
:10090000B5434560456896798E40B6B2354345603B
:10091000C5684F000326BE40B543C560D5794E007B
:10092000B540C6683543C560491C1029BFD3F0BD2A
:100930004FF6FF7101600021017141718171C17138
:10094000704708B54FF480320092009A0A43009233
:10095000009AC261C161009AC261C2690092C26913
:10096000009208BD0246002013690B400BB1012024
:1009700000E0002070470146086980B270470246D7
:10098000002053690B400BB1012000E000207047AC
:100990000146486980B270470183704741837047C0
:1009A0000AB1018300E041837047416170474269A9
:1009B0004A4042617047F0B5002300244D07ED0E18
:1009C00002FA05F3CE1000F1200555F826504E0727
:1009D000F70E0F26BE40B543CF1000F1200646F8B3
:1009E0002750CE1000F1200555F8265045EA0304A3
:1009F000CE1000F1200545F82640F0BD0000024071
:100A00000004024000080240000C024000100240B6
:100A10000014024000180240001C02400020024066
:100A20000024024000280240F948006840F001001C
:100A3000F74908600020F64908310860F44800686A
:100A4000F4490840F2490860F348091D0860F3487A
:100A5000EF4984310860F0481038091D0860EC48FF
:100A6000006820F48020EA4908600020E8490C3141
:100A70000860E7498C31086070470021E44A921C05
:100A8000117011460870704710B50146002200230E
:100A900000204A11012A02D1DD4C236808E0022A15
:100AA00003D1DB4C7034236802E0D94C74342368E2
:100AB00001F01F02012494401C400CB1012000E011
:100AC000002010BD38B5002000900024002500BF94
:100AD0003120FFF7D9FF05460098401C0090009890
:100AE000B0F5A04F01D0002DF2D03120FFF7CCFFA0
:100AF00008B1012400E00024204638BD0146002052
:100B0000C34A106820F0F80040EAC1001060704746
:100B1000C349086070470021BD4A703211701170DE
:100B2000012802D004280AD104E00121B84A703219
:100B3000117005E00521B64A7032117000E000BF67
:100B400000BF7047B7490860704770B5049C41EA20
:100B500082150126C6EB530645EA0645054345EADC
:100B60000465AB4E361D356070BDAD4908667047F3
:100B7000820142EA0172A64B84331A607047A84989
:100B80008866704710B5830143EA016343EA027344
:100B90009F4C8834236010BDA14908677047A04965
:100BA000C864704702460020994B0833186820F04B
:100BB000EC6042EA01031843954B08331860704714
:100BC00002460020924B0833186820F0784042EA31
:100BD000010318438E4B083318607047014600200C
:100BE0008B4A0832106820F00300084310607047F9
:100BF00087480830006800F00C007047014600206C
:100C0000834A0832106820F0F000084310607047F3
:100C1000014600207E4A0832106820F4E050084364
:100C20001060704701460020794A0832106820F4AD
:100C3000604040EAC10010607047F0B5002100221A
:100C40000024022500260223714F08373F6807F071
:100C50000C0121B1042905D0082937D105E0724FD4
:100C6000076036E0714F076033E0694F3F1D3F6812
:100C7000C7F38056664F3F1D3F6807F03F036EB1D4
:100C80006A4FB7FBF3F7DFF888C10CF1040CDCF80E
:100C900000C0CCF3881C07FB0CF40CE0624FB7FBE0
:100CA000F3F7DFF86CC10CF1040CDCF800C0CCF3F6
:100CB000881C07FB0CF4564F3F1D3F68C7F30147E4
:100CC0007F1C7D00B4FBF5F7076002E0564F07601C
:100CD00000BF00BF4E4F08373F6807F0F001090919
:100CE000534F7A5C0768D7404760494F08373F68E1
:100CF00007F4E051890A4E4F7A5C4768D740876015
:100D0000434F08373F6807F46041490B484F7A5C0E
:100D10004768D740C760F0BD002100F44072B2F5CB
:100D2000407F0AD13A4A0832116821F4F811414A49
:100D300002401143364A08321160354A7032126857
:100D4000C0F30B031A43324B70331A6070473549B6
:100D50004439086070473349403908607047364964
:100D60000860704701460020294A8C32106820F044
:100D70001F004A1E1043264A8C32106070470146FD
:100D80000020234A8C32106820F4F8504A1E40EAB2
:100D900002201F4A8C3210607047014600201C4A16
:100DA0008C32106820F440100843106070470146F0
:100DB0000020174A8C32106820F44000084310606D
:100DC000704701460020124A8C32106820F44030EF
:100DD00008431060704719490860704739B10C4AE0
:100DE0003032126802430A4B30331A6006E0084A78
:100DF000303212688243064B30331A607047F9B1C3
:100E0000034A343212680243014B34331A601CE047
:100E100000380240FFFFF6EA1030002400300020C6
:100E200000004742800E47420024F40000127A007E
:100E30001C000020FFFCFF0F5C014742E01147420D
:100E40008F4A126882438E4B1A60704739B18C4AC0
:100E5000121D126802438A4B1B1D1A6006E0884A65
:100E6000121D12688243864B1B1D1A60704739B1F0
:100E7000834A0C3212680243814B0C331A6006E03D
:100E80007F4A0C32126882437D4B0C331A607047E4
:100E900039B17B4A103212680243794B10331A6021
:100EA00006E0774A103212688243754B10331A609D
:100EB000704739B1724A243A12680243704B243B9E
:100EC0001A6006E06E4A243A126882436C4B243B57
:100ED0001A60704739B16A4A203A12680243684B77
:100EE000203B1A6006E0664A203A12688243644B4F
:100EF000203B1A60704739B1614A1C3A12680243BC
:100F00005F4B1C3B1A6006E05D4A1C3A1268824344
:100F10005B4B1C3B1A60704739B1594A143A12684E
:100F20000243574B143B1A6006E0554A143A1268C4
:100F30008243534B143B1A60704739B1504A103A00
:100F4000126802434E4B103B1A6006E04C4A103ABE
:100F5000126882434A4B103B1A60704739B1484AC5
:100F60001C3212680243464B1C331A6006E0444AA6
:100F70001C3212688243424B1C331A60704739B1ED
:100F80003F4A2032126802433D4B20331A6006E08C
:100F90003B4A203212688243394B20331A60704733
:100FA00039B1374A243212680243354B24331A6070
:100FB00006E0334A243212688243314B24331A60EC
:100FC000704739B12E4A2C32126802432C4B2C3315
:100FD0001A6006E02A4A2C3212688243284B2C33CE
:100FE0001A60704739B1264A303212680243244BE6
:100FF00030331A6006E0224A303212688243204BB6
:1010000030331A607047012808D11D493C31096806
:1010100041F008011A4A3C32116007E018493C319E
:10102000096821F00801164A3C321160704739B155
:10103000134A273A12780243114B273B1A7006E0F5
:101040000F4A273A127882430D4B273B1A7070479C
:101050000B484030006840F080700949403108601A
:10106000704701460020064A283A12680A400AB131
:10107000012000E0002070470149263908707047C0
:101080003438024010B50446FA48844208D10121A0
:101090001020FFF752FF00211020FFF74EFF57E00E
:1010A000F548844209D101214804FFF735FF0021AA
:1010B0004FF40030FFF730FF4AE0F048844209D196
:1010C00001218804FFF728FF00214FF48020FFF75B
:1010D00023FF3DE0EA48844209D10121C804FFF71B
:1010E0001BFF00214FF40020FFF716FF30E0E5481A
:1010F000844209D101210805FFF70EFF00214FF4BA
:101100008010FFF709FF23E0DF48844208D1012166
:101110002020FFF712FF00212020FFF70EFF17E02D
:10112000DA48844209D101218807FFF7F5FE002142
:101130004FF08040FFF7F0FE0AE0D548844207D127
:1011400001214005FFF7E8FE00216005FFF7E4FEFE
:1011500010BD2DE9FF4705460E460024A14600BFFD
:10116000A046B08900B100BF2C8A24F44054F08816
:1011700004432C82AC8941F20C608443B0883189ED
:101180000843718908430443AC81AC8A24F4407459
:10119000B0890443AC826846FFF74FFDB5488542ED
:1011A00002D0B948854202D1DDF80C9001E0DDF8AB
:1011B0000890A88900F4004040B109EBC90000EB99
:1011C000091031684900B0FBF1F707E009EBC900ED
:1011D00000EB091031688900B0FBF1F76420B7FB20
:1011E000F0F004012009642101FB1078A88900F4C3
:1011F000004040B1322000EBC800B0FBF1F000F03D
:101200000700044308E0322000EB08106421B0FB23
:10121000F1F000F00F0004432C81BDE8FF874FF48C
:101220001651016000218180C18001810C21418122
:1012300000218181704710B502460020108A20F4F9
:1012400070600B884C8823438C882343CC882343CD
:101250001843108210BD0021018041808180C1802F
:10126000704721B1828942F40052828104E0828970
:101270004DF6FF731A4082817047028B02F47F4261
:101280000283028B0A430283704721B1828942F4B0
:101290000042828103E08289C2F30E02828170479C
:1012A00021B1828A42F40062828204E0828A4FF293
:1012B000FF731A4082827047C1F308028280704730
:1012C00001468888C0F308007047028A4FF6F07321
:1012D0001A400282028A0A430282704721B182893F
:1012E00042F00202828104E082894FF6FD731A40C7
:1012F0008281704782894FF2FF731A40828182890E
:101300000A4382817047028A4FF6DF731A400282D5
:10131000028A0A430282704721B1028A42F4804263
:10132000028204E0028A4BF6FF731A400282704781
:10133000818941F001018181704721B1828A42F0A7
:101340000802828204E0828A4FF6F7731A40828292
:101350007047028BD2B20283028B42EA01220283DF
:10136000704721B1828A42F02002828204E0828AA0
:101370004FF6DF731A408282704721B1828A42F0B1
:101380001002828204E0828A4FF6EF731A40828252
:101390007047828A4FF6FB731A408282828A0A4320
:1013A0008282704721B1828A42F00202828204E086
:1013B000828A4FF6FD731A40828270471AB1838A7F
:1013C0000B43838202E0838A8B4383827047F0B5AC
:1013D0000346002400260025002040F66A17B94283
:1013E00000D100BF1846C1F3421401F01F060127C7
:1013F00007FA06F5012C01D10C3004E0022C01D1D2
:10140000103000E014301AB107682F43076002E083
:101410000768AF430760F0BD02460020B1F5007FCA
:1014200000D100BF13880B400BB1012000E0002069
:10143000704701F40072B2F5007F00D100BFCA43CB
:101440000280704770B5024600240023002500206A
:1014500040F66A16B14200D100BFC1F3421501F057
:101460001F03012606FA03F3012D13D19689334099
:1014700017E0000000100140004400400048004018
:10148000004C004000500040001401400078004033
:10149000007C0040022D02D1168A334001E0968A7A
:1014A00033400C12012606FA04F41688344013B1B6
:1014B0000CB1012000E0002070BD10B50022002317
:1014C00040F66A14A14200D100BF0A1201249440E0
:1014D000A3B2DC43048010BD002041490860091D0F
:1014E0000860091D0860091D08603E483C49143128
:1014F0000860704700213A498279002A3AD00A46AA
:10150000126803689A430B461A600A1D1268036842
:101510009A430B1D1A60027911440A6803681A4342
:101520000A602F4A0832126803689A432C4B08332A
:101530001A601A1D126803689A43294B0C331A600B
:101540004279102A0ED11A1F126803681A43244BDD
:1015500008331A601A1D126803681A43204B0C33B3
:101560001A600DE01E49427911440A6803681A4363
:101570000A6005E0027911440A6803689A430A6028
:1015800070470021016001710C21417100218171BE
:1015900070471349103109680143114A1032116034
:1015A0007047014600200E4A143212680A400AB100
:1015B000012000E00020704709491431086070479D
:1015C00001460020064A143212680A400AB101207E
:1015D00000E00020704702491431086070470000A5
:1015E000003C0140FFFF7F00FE4A1070704730B1A1
:1015F000FC49096841F48071FA4A116005E0F94933
:10160000096821F48071F74A1160704730B1F549DB
:10161000096841F40071F34A116005E0F149096875
:1016200021F40071EF4A1160704730B1ED4909684B
:1016300041F48061EB4A116005E0EA49096821F450
:101640008061E84A11607047E648006840F4006035
:10165000E44908607047E348006840F48050E1497D
:1016600008607047DF481030006800F0004028B183
:10167000DD48DC49091D0860DC4808607047D9482E
:101680001030006840F00040D649103108607047C3
:101690000920D4490C31096801F48031B1F5803F4B
:1016A00001D1012020E0CF490C31096801F010017F
:1016B00009B1062018E0CB490C31096801F48071AA
:1016C00009B1022010E0C7490C31096801F0EF01AF
:1016D00009B1072008E0C3490C31096801F0020193
:1016E00009B1082000E00920704708B509200090E2
:1016F000FFF7CEFF009002E0FFF7CAFF00909DF8D1
:1017000000000128F8D09DF8000008BD70B504461F
:101710000A460026092502B909E0012A01D116026C
:1017200005E0022A01D1160201E04FF44076FFF7EE
:10173000DCFF0546092D2DD1AA481030006820F4A1
:101740004070A849103108600846006830430860BE
:101750000846006820F0F80008600846006844F079
:10176000020108439F49103108600846006840F4B0
:1017700080300860FFF7B9FF05469A4810300068CE
:1017800020F002009749103108600846006820F0F8
:10179000F8000860284670BD30B5024600250924CF
:1017A000FFF7A3FF044602B909E0012A01D115029F
:1017B00005E0022A01D1150201E04FF44075092C21
:1017C00020D188481030006820F4407085491031DD
:1017D000086008460068284308600846006840F032
:1017E000040008600846006840F480300860FFF795
:1017F0007CFF04467B481030006820F004007949E3
:1018000010310860204630BD30B50246002509245D
:10181000FFF76BFF044602B909E0012A01D1150266
:1018200005E0022A01D1150201E04FF44075092CB0
:1018300020D16C481030006820F4407069491031A4
:10184000086008460068284308600846006840F0C1
:10185000040008600846006840F480300860FFF724
:1018600044FF04465F481030006820F004005D49E2
:1018700010310860204630BD30B5024600250924ED
:10188000FFF733FF044602B909E0012A01D115022E
:1018900005E0022A01D1150201E04FF44075092C40
:1018A00020D150481030006820F440704D4910316C
:1018B000086008460068284308600846006840F44D
:1018C000004008600846006840F480300860FFF778
:1018D0000CFF044643481030006820F400404149A2
:1018E00010310860204630BD70B5064614461D46CE
:1018F0000922FFF7FAFE0246092A1ED139481030A4
:10190000006820F4407037491031086008460068CC
:1019100040F4407008600846006840F0010008602C
:1019200034607560FFF7E1FE02462E481030006813
:1019300020F001002B4910310860104670BD30B511
:1019400002460C460925FFF7D0FE0546092D1DD19C
:1019500024481030006820F440702249103108609B
:101960000846006840F4007008600846006840F0CF
:10197000010008601460FFF7B8FE054619481030F2
:10198000006820F00100174910310860284630BD7A
:1019900030B502460C460925FFF7A7FE0546092D7E
:1019A0001DD110481030006820F440700D491031EE
:1019B00008600846006840F48070086008460068C7
:1019C00040F0010008601480FFF78FFE05460548CF
:1019D0001030006820F001000249103108602846EC
:1019E00030BD0000003C024023016745AB89EFCDCC
:1019F00030B502460C460925FFF777FE0546092D4E
:101A000017D19B48006820F4407099490860084647
:101A1000006808600846006840F001000860147023
:101A2000FFF763FE05469248006820F001009049E8
:101A30000860284630BD8E48001D006800F0010097
:101A400028B18C488A49083908608B48086070477B
:101A50008748001D006840F001008549091D0860A5
:101A6000704730B502460C460925FFF73EFE054695
:101A7000092D10D13CB17E48801D008890437C49DF
:101A8000891D088007E07A48801D008891B20843CC
:101A90007749891D088030BD30B502460C460925BE
:101AA000FFF723FE0546092D10D13CB170480A30DE
:101AB000008890436E490A31088007E06C480A307C
:101AC000008891B208436A490A31088030BDFF217D
:101AD000674AD21D127802F07F0140EA0102644B8E
:101AE000DB1D1A70704730B502460C460925FFF71A
:101AF000FCFD0546092D10D144B15D48801D0088CC
:101B000091B208435A49891D088006E05848801D53
:101B1000008890435649891D088030BD30B5024683
:101B20000C460925FFF7E1FD0546092D10D144B10A
:101B30004F480A30008891B208434D490A31088065
:101B400006E04B480A300088904349490A31088032
:101B500030BD10B502460924FFF7C7FD0446092C25
:101B600002D14348401D027010BDF0B504460D4639
:101B7000FF260927FFF7B9FD0746092F0BD13C487F
:101B8000001D007800F00F0645EA060010432043D0
:101B90003749091D0870F0BD3549091D097821F044
:101BA0001001334A121D117011460978014311705A
:101BB00070472F49091D097821F00C012C4A121D8C
:101BC00011701146097801431170704700B5092260
:101BD0002748001D007840F002002549091D0870C3
:101BE000FFF783FD0246104600BD2148001D006836
:101BF000C0F3471070471E48801D008870471C487E
:101C00000A30008870471A48801D008870471848BD
:101C10000A300088704700201549491D0978AA2913
:101C200001D0012000E0002070471148001D00781D
:101C300000F00C00704729B10D4A126802430C4BAA
:101C40001A6004E00A4A12688243094B1A6070471E
:101C500001460020064A121F12680A400AB10120FC
:101C600000E0002070470249091F0860704700002B
:101C7000103C02403B2A19087F6E5D4C00BF704744
:101C8000C2B2864B1A8000BF844A121F128802F02B
:101C90004002002AF8D0704770B504460D46294628
:101CA0002046FFF709FB00BF80212046FFF7B4FB69
:101CB0000028F9D070BD70B505460E46002404E03A
:101CC000295D7748FFF7E8FF641CB442F8D300BFF2
:101CD00040217348FFF7A0FB0028F9D070BD10B574
:101CE00088B0044601210846FFF778F8012110204A
:101CF000FFF7CEF8072209216A48FEF75CFE0722AB
:101D00000A216848FEF757FE4FF4C0600690022093
:101D10008DF81C008DF81D0000208DF81E0001209C
:101D20008DF81F0006A95F48FEF7BAFD0294002057
:101D3000ADF80C00ADF80E00ADF81000ADF81400D1
:101D40000C20ADF8120002A95548FFF702FA012154
:101D50005348FFF786FA40215148FFF76AFB0122FA
:101D600040F225514E48FFF732FB25208DF8040044
:101D700003208DF805008DF8060001208DF807007E
:101D800001A8FEF79CFC08B010BD10B588B0044651
:101D900001210846FFF722F801214804FFF767F800
:101DA000072202213F48FEF706FE072203213D4895
:101DB000FEF701FE0C20069002208DF81C008DF825
:101DC0001D0000208DF81E0001208DF81F0006A9BF
:101DD0003448FEF765FD02940020ADF80C00ADF824
:101DE0000E00ADF81000ADF814000C20ADF8120094
:101DF00002A92A48001FFFF7ACF901212748001F5C
:101E0000FFF72FFA40212548001FFFF712FB0122A0
:101E100040F225512148001FFFF7D9FA26208DF8FE
:101E2000040003208DF805008DF8060001208DF8D0
:101E3000070001A8FEF743FC08B010BD10B540F242
:101E400025511648001FFFF7FDFA30B31348001F55
:101E5000FFF736FAC4B21448008800F40040E0B935
:101E60000A2C01D00D2C06D10F48006840F4004028
:101E70000D49086011E00D480088C0F30D000C49C1
:101E80000C5409480068401C07490860084600686F
:101E9000B0F5806F01D30020086010BD04440040FD
:101EA0000010014000000240300000202C00002003
:101EB0008004002070B502464FF0FF30002410E08F
:101EC000155D80EA0560641C002308E000F0004511
:101ED0001DB1FD4D85EA400000E040005B1C082B71
:101EE000F4D30D1EA1F10101EAD170BDF8B506468B
:101EF0000F4639463046FFF7DDFF0546E8B28DF85C
:101F00000000280A8DF80100280C8DF80200280E28
:101F10008DF80300002404E0315DEC48FFF7BCFEBF
:101F2000641CBC42F8D3002405E01DF80410E74807
:101F3000FFF7B2FE641C042CF7D300BF4021E34836
:101F4000FFF76AFA0028F9D0F8BD2DE9F0470746F7
:101F50000C4614B90020BDE8F087DD480668FFF79D
:101F600081FB4FF0000800BF06F0010020B1761E93
:101F7000D84890F8009004E0404608F1010817F8AE
:101F80000090404608F10108385C49EA00294946BA
:101F90003046FFF7FDFCB61CA4EB08000228E3D294
:101FA000002509E0785DCA490968495D884201D089
:101FB0000120D0E7681C85B2A542F3D3FFF75FFB91
:101FC000C34800682044C24908600020C3E710B538
:101FD000FFF748FB02214020FFF798FB0221482031
:101FE000FFF794FBFFF74BFB10BD01460868BA4AA8
:101FF0001040B0F1005F01D1002070474FF0FF307A
:10200000FBE770B5044625682946B448FFF797FCFE
:1020100070BD70B50025B24CAC48FFF733F8B1483D
:102020000078012800D1B04C6568AE4803782A4694
:102030002146AEA000F0EEFABA480560206880F3B1
:10204000088800BFB7480068804770BD10B5B64823
:102050000078012806D002281CD01E2873D04428FE
:1020600072D140E00020B0490870B0480078B04913
:102070008871AE480088000AC871AC480068000C3E
:102080000872AA480068000E48720921A848FFF7A4
:102090002DFF5AE04FF40071A648FFF756FF0446A3
:1020A000012C03D1FFF793FF00F0E2F9A24800688A
:1020B00058B99E48006800F500709C4908600120EE
:1020C000994908709A4948710CE0984800689A4903
:1020D0000968084495490860442093490870032022
:1020E0009349487131E08048FFF77FFF40BBFFF71D
:1020F000B9FA02211020FFF709FB41F211118F48B4
:10210000FFF71DFCFFF7BBFA884800788849887103
:1021100086480088000AC87184480068000C08726C
:1021200082480068000E487209218148FFF7DEFEF0
:102130000220FEF76FFA01206A490870FFF769FF75
:1021400003E000E000E000E000BF00BF10BDF8B514
:102150007B480078002877D07A480079102806D08C
:1021600011280CD0122837D0FF286ED1FAE00120B8
:102170006F49487106217448FFF7B8FEF5E07148D1
:102180004079724908706F48807948706D48C0790D
:1021900088706C48007AC8706A48007B00066949FC
:1021A000C97A40EA01406749897A40EA01206549D5
:1021B000497A084366490860FFF709FF4A484449DD
:1021C00008600020594908605B49086001205649B1
:1021D000087060490870C8E05A48007A00065949FA
:1021E000C97940EA01405749897940EA01205549B7
:1021F000497940EA010658480068001F5149085CC7
:102200008DF8000054480068C01E085C8DF801007D
:1022100051480068801E085C8DF802004E48006836
:10222000401E085C8DF803004B480068011F4548BC
:10223000FFF740FE05460098A84234D13B480068AD
:10224000864230D1002408E095E08DE004F10900D9
:102250003C49085C37490855641CB4F5007FF5D348
:102260000220314908703C4800680D382F49096840
:1022700008443749096888421BD3374800680D383D
:102280002D49086008460068B0F5007F11D20A4663
:102290001268C2F50071274A274B1B68D018FF222D
:1022A00000F060FA05E001201F4908700220204973
:1022B00048710020294908600A20FEF7ABF9012087
:1022C0002749C1F8800250E0B71DC1040010014049
:1022D0004C000020780000200000FE2F00C0000805
:1022E0000000010800000020000008084A756D7019
:1022F0006164642069732025782C4A756D7041648F
:1023000064726573732069732025782C7570677209
:102310006164655F666C61672069732025640D0ADE
:102320000000000050000020700000206C00002021
:102330003E0000203C0B00207400002000800008BC
:10234000580000208008002038000020680000208D
:1023500054000020600000205C0000208082404289
:102360000080404200F084F800BF00BF00204849D0
:10237000086048490870F8BD10B540F2255146483C
:10238000FFF760F8002871D04348FEF799FFC4B208
:102390003F4801680068401C3D4A10603F48445473
:1023A0003C480078012803D13B48FEF789FF10BD67
:1023B0003B48007830B1012810D0022827D00328EC
:1023C00053D134E0A52C05D101203549087030499E
:1023D000086002E000202E49086046E05A2C0AD12D
:1023E000A5202E4908705A2048700220284908600C
:1023F0002B4908700AE0A52C05D101202849087056
:102400002349086002E00020254908702DE020489B
:10241000006804280AD3214880782049C97840EA16
:1024200001202049088003201D4908701DE01D4837
:102430000088B0F52F7F04DA15480068B0F52F7FCB
:1024400005D3002016490870114908600CE01548B2
:102450000088001D0E490968884205D801200D49F1
:10246000087000200E49087000BF00BF00BF9EE743
:10247000BFF34F8F0C48006800F4E0600B4908433D
:10248000001D09490860BFF34F8F00BFFEE7000041
:102490005C0000205800002000100140800800204F
:1024A000790000207A0000200CED00E00000FA0521
:1024B0001CB501210420FEF791FC122000900120A0
:1024C0008DF8040000208DF8060003208DF805002B
:1024D00001208DF8070069464748FEF7E1F912210F
:1024E0004548FEF759FA1CBD1CB501210220FEF734
:1024F00075FC40F20730009001208DF804000020A8
:102500008DF8060003208DF8050001208DF80700E6
:1025100069463A48FEF7C4F907213848FEF73CFA05
:102520001CBD704710B5FFF7FCFFFFF7DDFFFFF79D
:10253000BFFF10BD1CB501210220FEF74FFC4FF478
:102540008050009001208DF8040000208DF80600D6
:1025500003208DF8050001208DF807006946274803
:10256000FEF79EF90020264908603220FEF752F857
:1025700001202449C1F8B0023220FEF74BF80020B8
:102580001F4908603220FEF745F801201D49C1F8B7
:10259000B0023220FEF73EF81CBD1CB5012102201E
:1025A000FEF71CFC4FF44060009000208DF8040002
:1025B00003208DF8050000208DF8070069460F48BC
:1025C000FEF76EF91CBD10B54FF48060FEF7F8FF02
:1025D00028B101200C4908708002FEF7FCFF4FF47F
:1025E0000060FEF7EDFF28B1012008490870C00225
:1025F000FEF7F1FF10BD0000000802400004024099
:10260000B0824042008040427D0000207C000020DB
:10261000704700000FB4044910B503AA029800F0F7
:1026200007F910BC5DF814FB340000202DE9F041DF
:102630000E460446002020622046E168884730B3F9
:10264000252805D0D4E901219047206A401CF2E7F3
:10265000E168204600278847050018D0A5F1410011
:10266000192802D820354FF4006732462946204603
:102670002760FDF7C3FD40B1012804D0F61D26F008
:1026800007060836D8E7361DD6E72846DAE7206A77
:10269000BDE8F0812DE9F041064600241068752957
:1026A000314616A510D0AFF30080002802DA404270
:1026B00013A507E031688A0701D512A502E0490792
:1026C00004D511A5012401E0AFF3008000210A2206
:1026D00006F1240709E0B0FBF2FCB0FBF2F302FBC9
:1026E0001C00303078541846491C0028F3D123468A
:1026F0002A463046BDE8F04100F040B80000000036
:102700002D0000002B0000002000000070B50446E2
:102710000D4621461068AFF300802188090502D5D7
:102720000F4A7A4402E00E4A7A440E32002104F144
:10273000240305E000F00F060009965D5E54491C75
:102740000028F7D120780023000704D5702D02D08F
:1027500009B1022311322046BDE8704000F00EB8E6
:102760006802000002F0FF0343EA032242EA024249
:1027700000F072B870477047704770472DE9F04716
:102780000D4699469246044600F1240801688806E1
:1027900004D5E06921F01001216000E00120A84289
:1027A00001DD471B00E00027A1697A1902EB09004F
:1027B000081AA0612078C00602D42046AFF300803A
:1027C000002608E0D4E901211AF806009047206AA3
:1027D000401C761C20624E45F4DB2078C0060AD5EA
:1027E0002046AFF3008006E0D4E901213020904775
:1027F000206A401C2062381EA7F10107F4DC07E0C4
:10280000D4E9012118F805009047206A401C206295
:10281000281EA5F10105F3DC2046AFF300802078E7
:10282000000602D50220BDE8F0870120FBE700008A
:10283000074B70B50D467B4400F033F8044628463C
:1028400000F042F810B14FF0FF3070BD204670BD6F
:1028500047F4FFFF4FF000020429C0F0128010F08F
:10286000030C00F03780CCF1040CBCF1020F18BF50
:1028700000F8012BA8BF20F8022BA1EB0C0100F0FF
:1028800029B85FEAC17C24BF00F8012B00F8012BB6
:1028900048BF00F8012B704701694A1C02610878A3
:1028A000704700B58FB0CDE9013100210591054990
:1028B0007944CDE9031011466846FFF7B7FE0FB023
:1028C00000BD0000E5FFFFFF007B00F080007047C7
:1028D0004FF0000200B5134694469646203922BFB9
:1028E000A0E80C50A0E80C50B1F12001BFF4F7AF04
:1028F000090728BFA0E80C5048BF0CC05DF804EBE6
:10290000890028BF40F8042B08BF704748BF20F853
:10291000022B11F0804F18BF00F8012B704775464D
:1029200000F02CF8AE4605006946534620F007003B
:10293000854618B020B5FDF7ABFEBDE820404FF04E
:1029400000064FF000074FF000084FF0000B21F099
:102950000701AC46ACE8C009ACE8C009ACE8C00966
:10296000ACE8C0098D46704710B50446AFF300804F
:102970002046BDE81040FDF758BC000000487047F5
:102980003C0D00204FF04070E1EE100A70473031EE
:102990003233343536373839414243444546403086
:1029A0005800303132333435363738396162636438
:1029B0006566403078000000D8290008000000203B
:1029C00080000000C4010008582A00088000002090
:1029D00020130000E001000800000000007A030A54
:1029E00000000000000000000102030406070809BF
:1029F00000000000000000000102030401020304C3
:102A000006070809000000000000000000000000A8
:102A1000A55A06001001A55A0A0010000000000087
:102A200000000000000000000000000000000000A6
:102A30000000000000000000000000000000000096
:102A40000000000000000000000000000000000086
:082A500000000000000000007E
:040000050800018965
:00000001FF
